:020000020000FC
:1000000066C011C011C011C011C011C011C032C0F2
:1000100053C053C053C053C053C053C053C053C048
:1000200053C053C053C01895189518951895189536
:100030001FB71F934F935F93A8950CB95D9BFECF9D
:100040004CB95D9BFECF5FE75CB95D9BFECF22FFA5
:1000500005C0A0E6A0D09FD09ED0287F50E059BF19
:10006000C39B02C0C39801C0C39A5F914F911F9177
:100070001FBF18951FB71F930F93A8950CB120FDB4
:1000800006C00023A9F0A0E60D93206011C021FD59
:1000900003C00D9321600CC00C93539B02C02260DF
:1000A00007C0A0E6539A77D076D075D05398287FB2
:1000B0000F911F911FBF18951895189518951895B1
:1000C00018951895189518951895189518950FED79
:1000D0000DBF02E001BB0CE302BB0FEF07BB00EF5B
:1000E00008BB222700E034E0A6E60D933A95E9F735
:1000F000A0E60D930D930D9306E003B900E002B95D
:100100000FE109B908E90AB901E003BF00B3069598
:1001100006955FEF05270F70A02EA89509E001BD99
:10012000789400C0A895E6E6308143E2C79838D0BD
:10013000C79A31933081A895C69832D0C69A319328
:100140003081A895C5982CD0C59A31933081A89557
:10015000C49826D0C49A3083A89500B30695069516
:100160005FEF05270F70A02EDDCF0CE00A95F1F7A9
:10017000089500E90A0D5DEF52BF52E059BF00003B
:100180000000089500E80A0D5DEF52BF52E059BF2C
:100190000000000008950D910CB95D9BFECF0895FD
:1001A000439500E056B3587F050F08BBDEDF869904
:1001B00003C030FF04C008C030FD04C005C031607A
:1001C000D8DF02C03E7FDEDF439501E056B3587FA3
:1001D000050F08BBCADF869903C031FF04C008C001
:1001E00031FD04C005C03260C4DF02C03D7FCADFFC
:1001F000439502E056B3587F050F08BBB6DF8699DA
:1002000003C032FF04C008C032FD04C005C0346022
:10021000B0DF02C03B7FB6DF439503E056B3587FA3
:10022000050F08BBA2DF869903C033FF04C008C0D6
:1002300033FD04C005C038609CDF02C0377FA2DFF9
:10024000439504E056B3587F050F08BB8EDF8699AF
:1002500003C034FF04C008C034FD04C005C03061D1
:1002600088DF02C03F7E8EDF439505E056B3587F9E
:10027000050F08BB7ADF869903C035FF04C008C0AC
:1002800035FD04C005C0306274DF02C03F7D7ADFF7
:10029000439506E056B3587F050F08BB66DF869985
:1002A00003C036FF04C008C036FD04C005C030647A
:1002B00060DF02C03F7B66DF439507E056B3587F9F
:1002C000050F08BB52DF869903C037FF04C00895AD
:1002D00037FD04C0089530684CDF08953F7752DF42
:0202E00008957F
:00000001FF
